:020000040000FA
:020000000528D1
:06000A00031383128501BF
:1000100083163B30850053309F0083128501813069
:100020009F00831207309900A3018516A5209B200D
:100030007830C5000030C60023152630BA00B43031
:10004000B9009F111F15DA220030A8001B30A9004B
:10005000AB200310A70DA60D0310A70DA60D0310CE
:10006000A70DA60D0310A70DA60D0310A70DA60D35
:100070003430A900C2202608AC002708AD00483063
:10008000A900C2202608C7002708C8002C08A6001F
:100090002D08A7003830A900C2202608C90027086B
:1000A000CA004308A6004408A7000310A70DA60D28
:1000B000A8016430A900AB20F1224708A600480837
:1000C000A700F1224908A6004A08A700F122450826
:1000D000A6004608A700F12234214108A6004208E4
:1000E000A7004508A8004630A900B2205830CB0030
:1000F000AE21A61F842805114708C5004808C60080
:100100003030CB00AE218C2805154908C5004A08BF
:10011000C6003130CB00AE212C30CB00AE214108DF
:10012000A6004208A700F1220A30CB00AE210D3014
:10013000CB00AE211D287D30A00000000000000093
:1001400000000000A00B9D280800FA30A1009B20B1
:10015000A10BA72808002908A7070318A60A280842
:10016000A60708002908A702031CA6032808A60260
:100170000800A61FC128A609A7090130A707031870
:10018000A60A08002608AA002708AB00A601A701B6
:100190000730B000291FD42803102B08A707031C21
:1001A000D228A60A2A08A6070310AA0CAB0CA90D90
:1001B000B00BCA2808002310A310A61B2314A91BE8
:1001C000A314A61FE928A609A7090130A707031849
:1001D000A60AC22023080339033A0319FA28230880
:1001E0000339003A0319FA28A609A7090130A7071D
:1001F0000318A60A0800B9202608AC002708AD009D
:100200002808A6002808A700B9202608AE0027085D
:10021000AF002C08A6002D08A7002E08A8002F0864
:10022000A900B220A61B24292E08A6002F08A7008B
:100230000310A60CA70C0310A60CA70C2C08A800F2
:100240002D08A900AB2033292C08A6002D08A700F3
:100250000310A60CA70C0310A60CA70C2E08A800D0
:100260002F08A900AB200800B101B201B301B4010D
:10027000B501B601C830BB00BC019F111F11003091
:100280009000FE308F0046308E000C1010143308A2
:10029000B5003408B6003108B3003208B400CA21F2
:1002A0003C08A400D421BC0AA900A801C220260849
:1002B000B7002708B8003308A6003408A70039089B
:1002C000A900A801DB200310A70DA60D3508A80082
:1002D0003608A900B2203708A8003808A900AB20CA
:1002E0002608B1002708B2000C1C7429BB0B3F295B
:1002F0003508A6003608A7003908A900A801DB20A8
:100300002608A8002708A9003308A6003408A7007B
:10031000B2202608BD002708BE003508A600360812
:10032000A7003A08A900A801DB202608BF0027087B
:10033000C0003D08A6003E08A7003F08A8004008EE
:10034000A900FB202608C1002708C2000800000001
:100350003030CC000000CC0BAA2908000800851220
:100360000830CD00A72100000000000000004B1C59
:10037000BC2900008516BF29851200000000CB0CA7
:10038000A721CD0BB7290000000000000000851652
:10039000A72108009F149F18CB291E08A6008316CA
:1003A0001E088312A70008002408A500E030A50756
:1003B00001300318013E8A002508DF210800820071
:1003C0000534053405340534053405340634063463
:1003D0000634063407340734073408340834083444
:1003E000093409340A340A340B340B340C340C3419
:1003F0000D340E340E340F341034113411341234E1
:10040000133414341434153416341734183419349E
:1004100019341A341B341C341D341E341F34203458
:10042000213422342334233424342534263427340D
:10043000283429342A342B342C342D342D342E34C2
:100440002F3430343134323432343334343435347C
:1004500035343634373437343834393439343A343F
:100460003A343B343B343C343C343D343D343E340C
:100470003E343E343F343F343F343F343F344034E5
:1004800040344034403440344034403440344034CC
:10049000403440343F343F343F343F343F343E34C3
:1004A0003E343E343D343D343C343C343B343B34C8
:1004B0003A343A34393439343834373437343634DA
:1004C00035343534343433343234323431343034F6
:1004D0002F342E342D342D342C342B342A3429341B
:1004E0002834273426342534243423342334223446
:1004F000213420341F341E341D341C341B341A3470
:100500001934193418341734163415341434143497
:10051000133412341134113410340F340E340E34B9
:100520000D340C340C340B340B340A340A340934D3
:1005300009340834083408340734073407340634DF
:1005400006340634063405340534053405340534E0
:100550000408CE004F3084000530D400A401C4222A
:10056000A800A40AC422A900A40A8001B220A61BE4
:10057000BB2A800AB62AAB2030308004840AD40B10
:10058000AF2A4E08840008002408A500D030A50733
:1005900002300318013E8A002508CF22080082009D
:1005A000273410340334E8340034643400340A341B
:1005B00000340134A801A9010830A2009B20CA21FF
:1005C000AB202608A8002708A900A20BDE2A0310EA
:1005D000A60CA70C0310A60CA70C0310A60CA70CC6
:1005E0000800A8224F08CB00AE215008CB00AE2156
:1005F0005108CB00AE215208CB00AE215308CB00EE
:10060000AE212C30CB00AE2108002408A50011300B
:10061000A50703300318013E8A00250810230800AF
:1006200082003F343F343F343F343F343F343F3423
:100630003F343F343F343F343F343F343E343E3424
:100640003E343E343E343E343E343E343E343E341A
:100650003E343E343D343D343D343D343D343D3410
:100660003D343D343D343C343C343C343C343C3407
:100670003C343C343C343B343B343B343B343B34FF
:100680003B343B343A343A343A343A343A343A34F8
:1006900039343934393439343934393438343834F4
:1006A00038343834383438343734373437343734EE
:1006B00037343634363436343634363435343534EB
:1006C00035343534353434343434343434343434E7
:1006D00033343334333433343234323432343234E6
:1006E00032343134313431343134303430343034E4
:1006F00030342F342F342F342F342E342E342E34E4
:100700002E342D342D342D342D342C342C342C34E3
:100710002C342B342B342B342A342A342A342A34E4
:1007200029342934293429342834283428342734E6
:1007300027342734263426342634263425342534E9
:1007400025342434243424342434233423342334EB
:1007500022342234223421342134213420342034F0
:1007600020341F341F341F341F341E341E341E34F3
:100770001D341D341D341C341C341C341B341B34F8
:100780001B341A341A341A341934193419341834FD
:100790001834183417341734173416341634163402
:1007A000153415341434143414341334133413340A
:1007B0001234123412341134113411341034103410
:1007C00010340F340F340E340E340E340D340D3417
:1007D0000D340C340C340C340B340B340B340A341D
:1007E0000A34093409340934083408340834073425
:1007F000073407340634063405340534053404342C
:100800000434043403340334033402340234013432
:1008100001340134003400340034813481348134B3
:1008200082342408A5001D30A50704300318013EBA
:100830008A0025081C240800820082348334833413
:1008400083348434843484348534853485348634E4
:1008500086348734873487348834883488348934BC
:10086000893489348A348A348B348B348B348C3495
:100870008C348C348D348D348D348E348E348E346F
:100880008F348F3490349034903491349134913447
:100890009234923492349334933493349434943421
:1008A00094349534953496349634963497349734FA
:1008B00097349834983498349934993499349A34D4
:1008C0009A349A349B349B349B349C349C349C34AF
:1008D0009D349D349D349E349E349E349F349F3489
:1008E0009F349F34A034A034A034A134A134A13467
:1008F000A234A234A234A334A334A334A434A43441
:10090000A434A434A534A534A534A634A634A6341E
:10091000A634A734A734A734A834A834A834A934FB
:10092000A934A934A934AA34AA34AA34AA34AB34D9
:10093000AB34AB34AC34AC34AC34AC34AD34AD34B7
:10094000AD34AD34AE34AE34AE34AE34AF34AF3497
:10095000AF34AF34B034B034B034B034B134B13477
:10096000B134B134B234B234B234B234B234B33458
:10097000B334B334B334B434B434B434B434B4343A
:10098000B534B534B534B534B534B634B634B6341C
:10099000B634B634B734B734B734B734B734B83400
:1009A000B834B834B834B834B834B934B934B934E4
:1009B000B934B934B934BA34BA34BA34BA34BA34CA
:1009C000BA34BB34BB34BB34BB34BB34BB34BB34B0
:1009D000BC34BC34BC34BC34BC34BC34BC34BC3497
:1009E000BD34BD34BD34BD34BD34BD34BD34BD347F
:1009F000BD34BE34BE34BE34BE34BE34BE34BE3468
:100A0000BE34BE34BE34BE34BE34BF34BF34BF3453
:100A1000BF34BF34BF34BF34BF34BF34BF34BF343E
:100A2000BF34BF34BF34BF34BF34C034C034C0342B
:100A3000C034C034C034C034C0342408A5002930C8
:100A4000A50705300318013E8A002508282508005F
:100A50008200093409340A340A340B340B340B3461
:100A60000C340C340C340D340D340D340E340E347F
:100A70000E340F340F341034103410341134113458
:100A80001134123412341234133413341334143432
:100A9000143414341534153416341634163417340B
:100AA00017341734183418341834193419341934E5
:100AB0001A341A341A341B341B341B341C341C34BF
:100AC0001C341D341D341D341E341E341E341F349A
:100AD0001F341F341F342034203420342134213477
:100AE0002134223422342234233423342334243452
:100AF000243424342434253425342534263426342F
:100B0000263426342734273427342834283428340C
:100B100029342934293429342A342A342A342A34E9
:100B20002B342B342B342C342C342C342C342D34C7
:100B30002D342D342D342E342E342E342E342F34A7
:100B40002F342F342F343034303430343034313487
:100B50003134313431343234323432343234323468
:100B60003334333433343334343434343434343449
:100B7000343435343534353435343534363436342C
:100B80003634363436343734373437343734373410
:100B900038343834383438343834383439343934F3
:100BA00039343934393439343A343A343A343A34D9
:100BB0003A343A343B343B343B343B343B343B34BF
:100BC0003B343C343C343C343C343C343C343C34A6
:100BD0003C343D343D343D343D343D343D343D348E
:100BE0003D343D343E343E343E343E343E343E3477
:100BF0003E343E343E343E343E343E343F343F3463
:100C00003F343F343F343F343F343F343F343F344C
:100C10003F343F343F343F343F343F34403440343A
:100C20004034403440344034403440344034403424
:100C30004034403440344034403440344034403414
:100C40004034403440344034403440344034403404
:100C500040342408A5003530A50706300318013EAE
:100C60008A0025083426080082004034403440348D
:100C700040344034403440344034403440344034D4
:100C8000403440344034403440343F343F343F34C7
:100C90003F343F343F343F343F343F343F343F34BC
:100CA0003F343F343F343F343F343E343E343E34AF
:100CB0003E343E343E343E343E343E343E343E34A4
:100CC0003E343D343D343D343D343D343D343D349B
:100CD0003D343D343C343C343C343C343C343C3492
:100CE0003C343C343B343B343B343B343B343B348A
:100CF0003B343A343A343A343A343A343A34393484
:100D0000393439343934393439343834383438347E
:100D10003834383438343734373437343734373478
:100D20003634363436343634363435343534353476
:100D30003534353434343434343434343434333472
:100D40003334333433343234323432343234323470
:100D5000313431343134313430343034303430346F
:100D60002F342F342F342F342E342E342E342E346F
:100D70002D342D342D342D342C342C342C342C346F
:100D80002B342B342B342A342A342A342A34293471
:100D90002934293429342834283428342734273472
:100DA0002734263426342634263425342534253475
:100DB0002434243424342434233423342334223478
:100DC000223422342134213421342034203420347C
:100DD0001F341F341F341F341E341E341E341D3480
:100DE0001D341D341C341C341C341B341B341B3484
:100DF0001A341A341A34193419341934183418348A
:100E0000183417341734173416341634163415348E
:100E10001534143414341434133413341334123496
:100E2000123412341134113411341034103410349B
:100E30000F340F340E340E340E340D340D340D34A3
:100E40000C340C340C340B340B340B340A340A34A9
:100E500009340934093408340834083407340734B1
:0A0E60000734063406340534053467
:02400E00C230BE
:00000001FF
